:100000001AC3000035C3000033C3000031C3000031
:100010002FC300002DC300002BC3000029C3000024
:1000200027C3000025C300000C94E52C0C94CD2DB3
:100030000C949A2C1DC300001BC3000019C30000C0
:1000400017C3000015C3000013C3000011C3000054
:100050000FC300000C94C12C0BC3000009C30000A7
:1000600007C3000005C3000003C3000001C3000074
:10007000FFC20000FDC20000FBC20000F9C2000088
:10008000F7C20000F5C20000F3C20000F1C2000098
:10009000EFC20000EDC20000EBC20000E9C20000A8
:1000A000E7C20000E5C20000E3C2000005010980CC
:1000B000A101850319012AB700150126B700950192
:1000C00075108100C0050C0901A101850419012AE0
:1000D000A002150126A002950175108100C005013E
:1000E0000906A1018506050719E029E71500250184
:1000F0009508750181020507190029EF15002501F2
:1001000095F075018102050819012905950575010C
:100110009102950175039101C00660FF0961A1017B
:100120000962150026FF00952075088102096315F4
:100130000026FF00952075089102C005010906A15F
:1001400001050719E029E7150025019508750181CA
:10015000029501750881010507190029FF15002680
:10016000FF0095067508810005081901290515008D
:100170002501950575019102950175039101C00056
:10018000000000000000000000000000000000006F
:10019000000000000000000000000000000000005F
:1001A0000000007E0F00D4FFFFFFC70000007800B2
:1001B000000000000000002A2B28000000000000C2
:1001C0000000000000000000000029000000002CDA
:1001D0001E3420212224342627252E362D37382779
:1001E0001E1F202122232425263333362E37381F85
:1001F0000405060708090A0B0C0D0E0F1011121347
:100200001415161718191A1B1C1D2F3130232D35E4
:100210000405060708090A0B0C0D0E0F1011121326
:100220001415161718191A1B1C1D2F3130354C09BF
:10023000025B00030100A0FA0904000001030101B0
:100240000009211101000122440007058103080073
:10025000010904010002030000000921110100014D
:100260002222000705820320000107050303200066
:10027000010904020001030000000921110100012D
:10028000226D000705840320000112010002000016
:1002900000086A7001000100010203011C037600DE
:1002A000690061006C003A006600360034006300AB
:1002B000320062003300630000000E03540072003D
:1002C0006900700065006C0000000A0350006500C2
:1002D00065006A00000004030904240025002600CC
:1002E00027002A004C003400280018000C001200DF
:1002F000130033003800510052000D000E000F00B3
:100300003700360010004F005000167C1E001F0002
:10031000200021001500090019002B0014001A000C
:10032000080007000600E200E300E00004001600F9
:100330001B001D00E100E000215222002D005300AF
:100340002E0023001C000B00110017005F0060004E
:1003500061005E005B002C0000000A005C005D0094
:100360005A00590005000000000040004100420012
:1003700043004C00010001000100010001002F00BA
:100380003000010001000100010001000100010036
:100390000100010001000100010001003A003B00E2
:1003A0003C003D00010001000100010001000100CE
:1003B0000100010001000100010001000100010035
:1003C000010001000100010001003E004400450061
:1003D00068003F0001000100010001000100010070
:1003E0000100010001000100000001000100010006
:1003F0000100010001000000000001000100A30352
:100400005B12AF120000020002009F035B12AF12EA
:10041000000003000100A4035B12AF1200000400FF
:10042000020089035B12AF12040705000100A50357
:100430005B12AF120000060002008B035B12AF12CA
:10044000000007000200A1035B12AF1200001200BF
:100450000200A7035B12AF12000013000200A90301
:100460005B12AF12000014000100AB035B12AF126D
:1004700000001500000000000D07D40C000016005D
:100480000100A6037212C612000017000101A603A4
:100490007212C612000018000102A6037212C612E0
:1004A000000019000200AD035B12AF1200001A0039
:1004B0000103A6037212C61200001B000200AF0364
:1004C0005B12AF120000FD377A585A000004E6D6DE
:1004D000B4460200210116000000742FE5A3E002DB
:1004E0003400E65D003D8889C65436C3174FE4E406
:1004F000667274259658F24ED49CFC5234BA010EA2
:10050000A359AD51694215BD31C3FBD3D61F5DB7A9
:100510000423B5BD82726C40AF8FAF49C9D9201298
:100520008E3F251D7A533A6904C39F6FD245669D5D
:100530005BC24674DE142BB7534139DABA7A76F8C7
:10054000D8B77366F594B132A43C6B248B1C44324B
:10055000D9B191AA4EE4A2752D03EF932C4773579E
:100560001BFCD211A0A3A960B1A56208C0FA704B10
:10057000F08824CA37D003B881CAEB0B9C0EA19A2D
:100580003F983FAED8C266DCAE348151E6C7EBFF80
:1005900045032FF0FDDB10AC929DB659B88AE4F705
:1005A000885052664731ED6260C0A921ED382ADAE1
:1005B000298241A0C38D365508D0CDEE3E174D4E51
:1005C0000355717493EB8D438C7900000000446AED
:1005D0005BFB07B0412A00018202B50400001A2427
:1005E00048C7B1C467FB020000000004595A5252C8
:1005F00052525252525252525252525252525252DB
:100600005252525252524C4C4C4C4C4C4C4C4C4C06
:100610004C4C4C4C4C4C4C4C4C4C4C4C4C4C4C4C1A
:100620004C52525252524C4C4C5252522A004C4C48
:100630004C4C4C4C000011241FBECFEFDAE0DEBF63
:10064000CDBF11E0A0E0B1E0E0EFFEE502C0059013
:100650000D92AA3AB107D9F723E0AAEAB1E001C0A6
:100660001D92A63BB207E1F70E9406270C94E32EE9
:10067000C7CC9C019A9581159F4118F5F32FF27014
:10068000EE27832F8170732F74706627532F587055
:10069000442734FF0CC08295807FEF2B09F08062E5
:1006A000672B09F08064452B69F080680895EF2B73
:1006B00009F08260672B09F08460452B19F088608F
:1006C000089580E00895CF93DF93EB01D2DFFE0120
:1006D0000995DF91CF910895982F92959F7024E00E
:1006E000911102C020E0982F892F8695869581155B
:1006F00011F02E5F982F892F8695820F0895282F4D
:1007000092959F70963099F060F4925F9F7092304E
:1007100030F4203FB1F038F481E0283E38F080E03A
:1007200008959A5FF3CF81E0243FC9F7089591E0DF
:10073000813F09F090E081E0283E08F080E0892BBD
:10074000089581E0089580933D03089580933E03CA
:10075000089521E030E001C0220F8A95EAF78091E8
:100760003E03822BF3CF21E030E0A90102C0440F09
:10077000551F8A95E2F7CA01809590913E0389231F
:10078000E5CF993080F5883070F548E0949F90016E
:100790001124280F311D877041E001C0440F8A9554
:1007A000EAF783E0369527958A95E1F7F901EE0F90
:1007B000FF1FE20FF31FEC57FD4F80E090E070E069
:1007C0005191DF019B01082E02C0369527950A94AE
:1007D000E2F7217021952527242325272E930196C2
:1007E0008330910569F70895993078F5883068F578
:1007F00048E0949F90011124280F311D982F977085
:1008000083E0369527958A95E1F7F901EE0FFF1FF2
:10081000E20FF31FEC57FD4F40E050E080E02191E4
:1008200030E0092E02C0369527950A94E2F7217030
:100830003327042E01C0220F0A94EAF7822B4F5F60
:100840005F4F4330510559F7089580E00895909126
:100850003E0321E030E0F90101C0EE0F8A95EAF78E
:10086000D90102C0AA0FBB1F6A95E2F7EA2B01C0AB
:10087000220F4A95EAF7892F8E23E81303C0892FA8
:10088000822B64CF2095822F8923FBCF8091830216
:1008900090E020E0022E001C0008281709060CF04A
:1008A00008952F5FF7CFCF93DF93EC01DB018C81AD
:1008B000813059F514968C911497813031F5E98186
:1008C00088E0E89FF00111248881E80FF11DE251D2
:1008D000FA4F94919A32C9F01196EC91119788E0F1
:1008E000E89FF00111248C91E80FF11DE251FA4FBD
:1008F000E49181E09E1301C080E091E0EA3209F0CA
:1009000090E0892BDF91CF91089581E0FBCF9C018E
:1009100080913F038D79811119C0211540E534077D
:1009200080F4211580E23807C0F42333310511F13A
:10093000D0F481E02E31310590F42430310530F0CF
:100940000895C90196558115914010F080E00895F1
:10095000C901805F96450797C8F33327E6CF2C324D
:100960003105A1F708952653310981E0233031057F
:1009700038F3ECCF81E008958091490390914803CA
:10098000981301C008958F5F8770FACF9091430349
:100990008095892380934303282F2770211110C04D
:1009A000891771F09091B20392FF0AC086958695DF
:1009B0008695D9DE109243031092450310924403AA
:1009C000089590913F03982B90933F030895982F9B
:1009D000909580913F03892380933F0308958091F0
:1009E0003B03811531F010923B0310923A031092B1
:1009F00039030895803E9105D9F1C8F481339105FA
:100A000009F482C048F48932910509F472C08A322F
:100A1000910509F480C0089589339105E9F0823881
:100A20009105D1F08533910509F45EC00895843EA7
:100A30009105D9F148F4823E910539F1833E910543
:100A400049F181EE90E00895863E9105C9F1873E17
:100A5000910509F43EC008952091B103237021113E
:100A600064C02091B20323FF14C089E290E008958E
:100A70002091B10320FD45C03091B20330FF09C081
:100A800024FD24C083EE90E008952091B10322FD5F
:100A9000F7CF08952091B10322FD44C03091B203F5
:100AA00030FD43C024FFF5CF11C02091B20321FFD8
:100AB000F0CF8091B10384FD09C087EE90E00895E6
:100AC0002091B10323FFE5CF24FFF7CF80E090E032
:100AD00008952091B10323FD2BC03091B20331FF63
:100AE000E1CF84EE90E008952091B10325FFD1CFAE
:100AF000BCCF2091B10325FD1EC02091B20323FF7E
:100B0000C8CF89E390E008952091B10326FFC1CFBB
:100B10008AE290E008952091B10326FFBACF81E3E5
:100B200090E0089582EE90E0089580EE90E00895C0
:100B300086EE90E0089585E390E008959091B103EA
:100B400092FF10C041E0282F2471243009F040E0CA
:100B500031E0282F2871283009F030E0431711F0D8
:100B60002CE0822793FF10C041E0282F247124310C
:100B700009F040E031E0282F2871283109F030E0F9
:100B8000431711F02CE082273091B20330FF10C0E0
:100B900051E0282F2171213009F050E041E0282F49
:100BA0002871283009F040E0541711F029E082271D
:100BB00031FF10C041E0282F2171213109F040E0C0
:100BC00031E0282F2871283109F030E0431711F067
:100BD00029E0822794FD877E08951F93CF93DF93AA
:100BE00009DFEC01811522E5920708F052C081155A
:100BF00040E5940708F0CDC0803E910520F58D3C7E
:100C0000910508F0A1C0883A910570F4853A9105E4
:100C100008F097C081309105B9F10497813A9105A8
:100C200098F1C0E0D0E030C0885A91094B97C8F7DE
:100C3000C85AD0E0CC0FDD1FC25CDE4F0990D881CE
:100C4000C02DD46421C0811550E49507B0F4C115BE
:100C500080E2D80708F0B3C0C83ED105A8F0CE01A5
:100C60009A9581159F41E8F68D2F68DF182FCE01E8
:100C70009927C0DEEC01D12B07C09927BBDECC271A
:100C8000DF70C82BD92BD06ACE01DF91CF911F9195
:100C90000895803842E59407C8F5803652E59507F7
:100CA00008F05BC0C03482E5D807D0F4C03292E5CA
:100CB000D90708F04BC08C2F8695869520E2829F3D
:100CC000C0011124C37021E030E0A90102C0440F2B
:100CD000551FCA95E2F7EA01C82BD92BDD68D4CF9E
:100CE0008C2F86958695877050E2859FC0011124D0
:100CF000C37021E030E0A90102C0440F551FCA951E
:100D0000E2F7EA01C82BD92BDC68BECF803C52E564
:100D1000950758F48F71C03AD245A0F590E0982F0E
:100D20008827EC01C46FD06AAFCF805C9245809772
:100D300008F077CFDC2FCC27CC27DF71C06FD06ACB
:100D4000A3CFA497D064A0CFD0659ECFCF71D0E0C1
:100D5000DC2FCC27C16FD06A97CF86958695877098
:100D600020E2829FC0011124C37021E030E0A9017C
:100D700002C0440F551FCA95E2F7EA01C82BD92BD0
:100D8000DA6882CFDBDEC82FD0E0DC2FCC27D06240
:100D90007BCF8F71D3DE93E0CC0FDD1F9A95E1F707
:100DA000CC27DF70282F30E084FF05C050E1859FFD
:100DB000900111243327C22BD32BD06965CF8D2FFF
:100DC0008F71BCDE182FCE01992714DEEC01D12BD8
:100DD000DECF80E00895F894E82FE295EF70F0E020
:100DE00041A18F7021E030E0B90102C0660F771F8A
:100DF0008A95E2F7CB01962F9095942391A392A127
:100E0000892B82A3789408958091890390918A0315
:100E100090930D0180930C010895EF92FF920F9330
:100E20001F93CF93DF93FB018FEF9FEF443051056A
:100E300008F45FC04091B10341FB882780F990E03E
:100E4000880F991F42FB002700F910E0000F111FC7
:100E5000000F111F802B912B40FBEE24E0F8F12CAA
:100E60008E299F2943FB222720F9C22F50E0D52F3E
:100E700053E0CC0FDD1F5A95E1F78C2B9D2B44FBE3
:100E8000222720F950E1259F90011124822B932BDA
:100E900045FB222720F950E2259F90011124822B47
:100EA000932B46FB222720F950E4259F9001112423
:100EB000822B932B47FB222720F940E8249F9001A7
:100EC0001124822B932B2091B203322F3170932B5C
:100ED00026952170B22FBB0FA0E08A2B9B2B092EE9
:100EE000000CAA0BBB0B80839183A283B38380E0A9
:100EF00090E0CDB7DEB7E6E00C94402EAC0123E0E5
:100F0000969587952A95E1F78E719927FC01EC500B
:100F1000FE4F0190F081E02D4F70552721E030E029
:100F200002C0220F331F4A95E2F7611541F0E22B10
:100F3000F32B8C509E4FDC01ED93FC93089520958C
:100F40003095E223F323F5CFFC01848186238111C0
:100F50000AC082818115B9F06823908593FF05C08E
:100F600081E061110FC080E00895282F22952F7035
:100F70008F70282B962F92959F706F70962B81E023
:100F80002913F1CF089581E008950F931F93CF9314
:100F900001E010E0082E01C0000F0A94EAF7C091AA
:100FA00038039C2F9023911115C09091430396957F
:100FB00096959695891306C01092430310924503A7
:100FC00010924403C6DBC027C0933803CF911F9112
:100FD0000F910895C8DBF7CFE0916902F0916A02A2
:100FE000309739F00190F081E02D309711F009959C
:100FF000089580E00895A3E0B0E0E1E0F8E00C940B
:10100000282E9C018091F2019091F30182179307A1
:10101000B1F03093F3012093F201E0916902F09175
:101020006A02309761F00084F185E02D309739F045
:1010300083E089833B832A83CE0101960995239619
:10104000E2E00C94442EA3E0B0E0E9E2F8E00C9476
:10105000282E9C018091F0019091F1018217930755
:10106000B1F03093F1012093F001E0916902F09129
:101070006A02309761F00084F185E02D309739F0F5
:1010800084E089833B832A83CE01019609952396C8
:10109000E2E00C94442E90911001913091F0AEEA70
:1010A000B1E0EFEF90E02D91821751F0EF3F19F48E
:1010B000211101C0E92F9F5F9630A9F7EF3FC9F4D6
:1010C00008959091B10397FFEACFE82FE695E69552
:1010D000E695803FA8F7F0E0EC54FE4F877021E0E2
:1010E00030E001C0220F8A95EAF78281822B828349
:1010F00008950E2E000CFF0BE455FE4FF8CF909193
:101100001001913021F49091B10397FD0CC0EEEAEB
:10111000F1E09191891302C0DF011E9251E0E43B9E
:10112000F507B9F70895E82FE695E695E695803F2F
:10113000C8F7F0E0EC54FE4F877021E030E0A901E1
:1011400002C0440F551F8A95E2F7CA01809592812B
:1011500089238283089580910F0108952FB7F89411
:101160008091EC019091ED01A091EE01B091EF0121
:101170002FBF089580918B0390918C03892B89F068
:10118000EDDF2091390330913A03AC01421B530B40
:101190009A0181E040918B0350918C03241735070D
:1011A00008F480E00895CF93DF93C0913F038091CE
:1011B0004203C82B80913B038115E1F080918B03A2
:1011C00090918C03892B19F0D5DF811108DCD09127
:1011D0003B0380911001813021F48091B10387FDA0
:1011E00013C086E02EEA31E090E0815088F491113E
:1011F000F6DBCD2B8091A70280958C239091A602DF
:10120000892BDF91CF9108958EE126EB31E0ECCF71
:10121000F90141919F01411541F39F5FE6CF962F60
:101220002091B20322FF0EC0682F660F660F660F73
:10123000692B609343038DDA91DF9093450380938C
:101240004403089586CA90913B03292F2823211532
:1012500059F08095892380933B03811531F07EDF1F
:101260008093390390933A03089580E090E0F8CF9B
:10127000CF93C82F8091B20382FF0BC080913B03B4
:101280008C1739F06BDF90933A0380933903C09346
:101290003B03CF9108952FB7F8946091EC017091C2
:1012A000ED018091EE019091EF012FBF0895CF9253
:1012B000DF92EF92FF92CF93DF93D82FC92FC09088
:1012C0002503D0902603E0902703F0902803E3DF66
:1012D0006C197D098E099F09643F71408105910554
:1012E00010F1D9DF6B017C0182E390E0A0E0B0E077
:1012F000C0922E02D0922F02E0923002F092310280
:1013000080932A0290932B02A0932C02B0932D027B
:10131000D0932303C0932403DF91CF91FF90EF90EC
:10132000DF90CF90089584EF91E0A0E0B0E0E0CFAF
:1013300087E797E7909301088093000888E19AE097
:101340000FB6F894A895809360000FBE909360004C
:10135000FFCF0895FC019B018091E2019091E30190
:101360008617970740F0672B29F48091E8008E7765
:101370008093E800C90140E0009741F4411106C0A4
:101380008091E80082FF2FC080E008952091420202
:101390002115A9F12530A9F12091E80023FD2DC0E8
:1013A0002091E80022FDECCF2091E80020FFE4CF5F
:1013B0003091F3002091F200009719F028303105A8
:1013C00058F041E02830310509F040E02091E80074
:1013D0002E772093E800D0CF41914093F100019700
:1013E0002F5F3F4FE9CF80914202811541F0853058
:1013F00041F08091E80083FFC3CF81E0089582E04F
:10140000089583E008958091DC0187FF13C08091E7
:10141000E80082FF06C08091E8008B778093E800A7
:101420000895809142028111F2CF08958091420285
:101430008115D9F38091E80080FFF8CF8091E80012
:101440008E77ECCF2091E4003091E50095E6A9017C
:101450002091EC00822F817020FF06C08091E8006F
:1014600080FF06C080E008952091E80022FD1AC0A8
:1014700080914202811589F0853089F08091EB00DE
:1014800085FD0FC02091E4003091E500421753071D
:10149000F9F29A95E1F684E0089582E0089583E0F8
:1014A000089581E00895E8EDF0E080818E7F8083EB
:1014B0001092E2001092DA001092E100A0EEB0E08B
:1014C0008C9181608C9380818F77808319BCA7ED8C
:1014D000B0E08C918E7F8C9380818F7E8083109280
:1014E000DB010895E0916902F0916A02309739F0CA
:1014F0000284F385E02D309711F060E2099508959C
:10150000982F9093E900891771F07091EC00209169
:10151000ED005091F00021FD09C09F5F973089F7E1
:101520008093E9000895762F242F50E03091EB004E
:101530003E7F3093EB003091ED003D7F3093ED0026
:101540003091EB0031603093EB007093EC0020930E
:10155000ED005093F0002091EE0027FDDECF0895BE
:10156000A0E0B0E0E6EBFAE00C94222EC8EDD0E06B
:1015700088818F7E8883E7EDF0E0808181608083C1
:1015800084E082BF81E08093DB0188818E7F888345
:1015900002EE10E0F80110821092DA0081EEC82EFF
:1015A000D12CF601108288818F77888388818068AA
:1015B000888388818F7D888319BC109242021092A3
:1015C000DA0110921F021092D90190EEE92EF12C4F
:1015D000F70180818B7F808388818160888342E0EE
:1015E00060E080E08DDFF60180818E7F8083F801EE
:1015F000808181608083808188608083F701808121
:101600008E7F8083888180618883CDB7DEB7E8E0F4
:101610000C943E2EE09149039091480327E0E91392
:1016200002C080E00895AE2FB0E02E9FF00111249B
:10163000E65BFC4F3181361306C03081381303C09E
:101640003581341304C0FD013196E770E8CF81E0A5
:1016500008959C012115310509F408958FE99FE053
:101660000197F1F700C0000021503109F3CF0F932B
:101670001F93CF93DF938B01EA0190914202943044
:1016800051F58093E9008FEF9091E80095FD06C039
:1016900095ED9A95F1F700008A95B1F78091E800F1
:1016A00085FF19C0CFDE811111C08091E80085FD52
:1016B00006C08091E8008E778093E800F3CFF801B0
:1016C00081918F018093F100219779F78091E80053
:1016D0008E778093E800DF91CF911F910F9108954D
:1016E000792F603229F440E250E0682F82E0BFCFCA
:1016F0000895CF93DF93D82FC92F48E050E0682F8B
:10170000792F81E0B4DF88E0ED2FFC2FA4EEB1E06B
:1017100001900D928A95E1F7DF91CF910895BC0178
:1017200040E250E084E0A3CFBC0143E050E084E01D
:101730009ECFFC016081718184E090E00C94C82E02
:101740009091B20392FB222720F9281749F080FBE1
:1017500092F99093B20381EB93E0EBDF82E016C93C
:1017600008951F93CF93DF93C62F122F632F8430DA
:10177000D0F4C930C0F44830B0F490E1C99FE00122
:101780001124C40FD11DC40FD11D90E9899FC00D34
:10179000D11D1124CE0189960E94AE2E612FCE015B
:1017A0008A960E94AE2EDF91CF911F91089580916D
:1017B0001001813061F58091B10387FF28C0F3DC0F
:1017C0008093B50140E250E069E472E084EB91E07F
:1017D0000E94652E892BD1F080E2E4EBF1E0A9E4D0
:1017E000B2E001900D928A95E1F7E0916902F091E3
:1017F0006A02309759F00480F581E02D309731F07E
:1018000086E08093B40184EB91E009950895CBDCE8
:101810008093AC0148E050E06BE672E08CEA91E026
:101820000E94652E892B91F388E0ECEAF1E0ABE6AB
:10183000B2E001900D928A95E1F7E0916902F09192
:101840006A02309719F30280F381E02D3097F1F2AC
:101850008CEA91E0DACF811511F0B3D8A8CF0895C2
:10186000811531F090914203892B809342039FCFE1
:101870000895811511F0ABD89ACF0895811539F0EC
:1018800080959091420389238093420390CF0895DD
:101890008091A202811521F082E2F0DF1092A20273
:1018A0000895811501F19CEF980F913A10F427DC0F
:1018B0007ECF90E2980F983048F4877091E001C095
:1018C000990F8A95EAF7892F82D8F2CF9BE5980F76
:1018D000933018F480E090E08ECB885A8B3118F466
:1018E00080E090E0B0CB0895CF93DF93EC01D9DF97
:1018F000CE01805E9109089720F06EE37CE020978E
:1019000011F469E37CE0CE010E946303DF91CF9183
:10191000089510923F03809110018130A1F48091CD
:10192000B10387FF10C0E6EBF1E08EE1DF011D920D
:101930008A95E9F780E090E05EDB80E090E083DB71
:101940001092420334CFEEEAF1E086E0EFCFE1DF20
:101950002FEF84E39CE0215080409040E1F700C0ED
:10196000000088E19AE00FB6F894A8958093600093
:101970000FBE90936000FFCFCF93DF93D82FC92F76
:1019800020918302283010F0C4DF20E0E22FF0E045
:10199000EE0FFF1FED58FD4FD083C1832F5F2093C3
:1019A0008302DF91CF910895CF93DF93FB018FEFF7
:1019B0009FEF4430510588F0D081C181AADFD093D8
:1019C000B103C3708091B2038C7FC82BC093B20364
:1019D00081EB93E0AEDE80E090E0DF91CF9108955F
:1019E000AAE2B0E0E6EFFCE00C94272E8CED91E04B
:1019F000FC0101962091F100208321E0843E9207B2
:101A0000B9F78091DD01893009F457C0C8F48230FC
:101A100009F4B2C0833009F482C0813081F1809131
:101A2000E80083FFE6C08091DC019091DD019A30EF
:101A300008F0DFC0E92FF0E0EB51F14D0C944F2E90
:101A40008A3009F489C08B3051F78091DC018132F2
:101A500031F78091E0019091E101892B01F78091AC
:101A6000E800877F8093E800CEDC81E09091DE0182
:101A7000911101C080E0809310014BDFD0CF8091A5
:101A8000DC01813A61F68091E800877F8093E8006D
:101A90008091E0019091E101892B59F060E080E0B4
:101AA00090E070E057DC8091E8008B778093E8004D
:101AB000B6CF68E084EE91E0F4CF8091DC01813212
:101AC00009F0ADCF8091E0019091E1018D7F892BEC
:101AD00009F0A5CF8091E800877F8093E80080918E
:101AE000E80082FF17C09091F3008091F200029706
:101AF00031F48091F100813011F0863021F4809131
:101B0000F10080930F018091E8008B778093E800CB
:101B10007ADC85CF809142028111E1CF80CF809124
:101B2000DC01813A09F07BCF8091E0019091E101E5
:101B3000892B09F074CF8091E800877F8093E800BB
:101B40008091E80080FFFCCF809110018093F1002C
:101B50008091E8008E77DACF8091DC01813209F044
:101B60005ECF8091E800877F8093E8004CDC809115
:101B7000DF0180930E0153CF8091DC01813A09F09F
:101B80004ECF8091E800877F8093E8008091E80045
:101B900080FFFCCF80910E01D9CF803889F0823848
:101BA00041F58091E0018F70873018F58093E9004E
:101BB0008091EB0085FB882780F91092E90006C030
:101BC00080911F02880F9091D901892B9091E80094
:101BD000977F9093E8008093F1001092F10080913C
:101BE000E8008E7723C0811116C08091DE0181301C
:101BF00009F18091E80083FF0AC08091E800877FA7
:101C00008093E8008091EB0080628093EB00AA96BD
:101C1000E3E00C94432E823061F78091DE01811560
:101C200081F01092E9008091E800877F8093E800BE
:101C3000EADBDFCF81E0933009F080E080931F0280
:101C4000F0CF8091E0018F702FEF280F263088F6BB
:101C50008093E9002091EB0020FFE3CF933031F433
:101C60008091EB0080628093EB00DBCF9091EB00E2
:101C700090619093EB0021E030E0A90102C0440F95
:101C8000551F8A95E2F74093EA001092EA0080918E
:101C9000EB008860E8CF8111ACCF1091DE011F7797
:101CA0008091E3008078812B8093E3008091E800AD
:101CB000877F8093E800A7DB8091E80080FFFCCF5E
:101CC0008091E30080688093E30083E0111101C0FC
:101CD00082E0809342028DCF8058823008F089CF15
:101CE0008091DE019091DF018C3D53E0950791F5E5
:101CF00083E08A838AE289834FB7F894DE011396E2
:101D000020E03EE051E2E32FF0E050935700849151
:101D100020FF03C082958F703F5F8F708A30C0F0C4
:101D2000895C90E08D939D932F5F243161F74FBFC5
:101D30008091E800877F8093E8006AE270E0CE013E
:101D4000019608DB8091E8008B778093E80051CF03
:101D5000805DE7CF292F33272330310509F44EC0AA
:101D600078F52130310509F488C08BE590E0EFE289
:101D7000F2E02230310509F03CCF2091E800277FC6
:101D80002093E8002091E2013091E301821793074C
:101D900008F49C0140E02115310509F073C04111A0
:101DA00071C08091E80082FDCDCF80914202811503
:101DB00049F2853039F28091E80083FFF2CFC2CF3B
:101DC0008091E0019091E1012132310509F446C092
:101DD0002232310509F00DCF8330910508F009CF8B
:101DE000FC01EE0FFF1FEF5DFE4F0190F081E02D33
:101DF000825E9E4FDC018C9190E010C09C013327E5
:101E0000823021F12330310568F4232BB9F4E6ED5B
:101E1000F2E0E4918E2F90E0E6EDF2E0009709F415
:101E2000E8CEABCF2330310509F0E3CEECE9F2E0A8
:101E3000E4918E2F90E0ECE9F2E0F0CFEAECF2E0F2
:101E4000E4918E2F90E0EAECF2E0E8CFEAEBF2E0EA
:101E5000E4918E2F90E0EAEBF2E0E0CF8330910541
:101E600008F0C7CEFC01EE0FFF1FE95DFE4F0190A9
:101E7000F081E02D89E090E080CF82E190E0EAE817
:101E8000F2E07BCF80914202811509F45BCF85306F
:101E900009F458CF8091E80083FD54CF8091E80089
:101EA00082FD7FCF8091E80080FF75CF9091F30095
:101EB0008091F2002115310519F08830910550F01C
:101EC00041E0089709F040E08091E8008E77809328
:101ED000E80061CF44914093F100319621503109DF
:101EE0000196E8CF803809F084CE8091E800877FA2
:101EF0008093E8008091DA018093F10070CE811127
:101F000078CE1091DE01123008F073CE8091E80097
:101F1000877F8093E8001093DA0175DA1115D9F004
:101F200084E08093420242E061EC81E0E9DA42E23F
:101F300061EC84E0E5DA42E261EC82E0E1DA42E27F
:101F400060EC83E0DDDA80914202843051F482E07B
:101F5000809311014ECE8091E30087FDE1CF81E0B7
:101F6000E0CF81E0F5CF80911301877F809313014B
:101F70008091A202811105C0809142038D7F8093E0
:101F800042038091130184FF06C08F7E809313016A
:101F900082E00E94E1048091130185FF06C08F7DDD
:101FA0008093130180E20E94E10401CC1F93CF9340
:101FB000DF93182FA0912103B0912203109709F409
:101FC00047C010922403109223031092A70210928C
:101FD000A6021696CD91DC911797CE019A958115A0
:101FE0009F4108F4D07ED1E0C11101C0D0E0199624
:101FF000ED91FC911A97309731F01B966D917C9181
:1020000080E00995D823D11531F08CEF8C0F813AFF
:1020100018F58C2F74D81115A1F0E0912103F091DF
:102020002203808584FD0DC080912003811549F035
:10203000808191819C01215031092F333E4708F462
:1020400036D9B5DB1092220310922103109220039F
:10205000DF91CF911F910895AADB8C2F22DCDBCF7B
:102060000F931F93CF93DF9309E813E0C9E6D2E003
:10207000CE010E94922EF80161918F01681719F02C
:10208000CE010E94AE2E2196C139F2E0DF0781F722
:10209000DF91CF911F910F9108950F931F93CF93CD
:1020A000DF9309E813E0C9E6D2E0CE010E94922E48
:1020B000F80181938F012196C139F2E0DF07A9F77A
:1020C000C4E0D4E0FE0185919591009711F0FC01E8
:1020D00009952C96F4E0C03DDF07A1F7DF91CF9181
:1020E0001F910F910895E9E8F3E0128E138E8FEAA5
:1020F00090E09183808385E0848F28E833E1338307
:10210000228322E330E0378B268B28EC30E0318FBE
:10211000208F158E35A324A3178E168E20E530E070
:1021200031A320A382A317A216A29ADFF2DB10929A
:10213000B2031092B10380E084608093B20381EB1C
:1021400093E0F7DAAACF0F931F93CF93DF938430F6
:1021500028F5693018F5483008F520E1629FE00164
:102160001124C40FD11DC40FD11D30E9839FC00DB0
:10217000D11D1124CE0189960E94922E082F10E0C5
:10218000102F0027CE018A960E94922E9801282BAC
:10219000C901DF91CF911F910F91089580E090E0E8
:1021A000F8CF462F672F2091450230914602232B0E
:1021B00081F4703F39F4403F61F480914302909183
:1021C00044020895793028F4483018F4843008F433
:1021D000BACF80E090E00895A0E0B0E0E2EFF0E157
:1021E0000C94232E7C0100913E0380913D03082B2B
:1021F000C3E0D0E010E0C8010C2E02C09595879591
:102200000A94E2F780FD09C02197A8F7D12C8D2D03
:10221000CDB7DEB7E7E00C943F2EDC2EB7018C2F54
:10222000C0DF0E94ED05019779F3F1CFCF93DF93E3
:10223000D82FC92FD1DF6D2F7C2FB3DF0E94ED0582
:10224000DF91CF910895FC018481811529F080816F
:102250009181ECDF0C947F0380E008951F93CF936E
:10226000DF93182FD92F611589F0411579F0B4DF6C
:10227000C82F682F812F9D2F0E94C103612F7D2FB2
:102280008C2F8FDFDF91CF911F9108950E94F4036F
:10229000C82FF4CFFC01462F658180819181DECF6C
:1022A000382F292FCB01A32FB22F8F3121E0920796
:1022B000A105B10520F48F519D4F0C94922E80E022
:1022C000089585E290E00E94922E863289F486E29B
:1022D00090E00E94922E863E59F487E290E00E94A0
:1022E000922E91E0803409F090E0892F817008955A
:1022F00080E0FCCFAAE0B0E0E0E8F1E10C94202E11
:1023000008EA12E081E9E82E82E0F82E97E0B92E83
:1023100024E1C22E22E0D22EAA24A3944AE050E067
:10232000B701CE0101960E94822EF8013896DF0196
:102330008B2D1D928A95E9F789819A81D801119692
:102340009C938E938F8112968C9312978D81139606
:102350008C931397888514968C931497898515967A
:102360008C9315978B819C8117969C938E931697CF
:102370008A8587FD04C01E96DC92CE921D9780FF51
:1023800002C0F801A08681FF07C0D80118969C9171
:102390001897926018969C9382FF04C0F80190856C
:1023A0009460908783FF07C0D80118969C91189776
:1023B000986018969C9384FF04C0F8019085906102
:1023C000908785FF07C0D80118968C911897806276
:1023D00018968C93BAE0EB0EF11C015F1F4FE1EEF3
:1023E000EE16E2E0FE0609F099CF2A96EAE00C9498
:1023F0003C2EAAE0B0E0EFEFF1E10C941D2EA0908E
:102400004002B090410281E090E0909341028093BD
:102410004002812C912C00E0640110E019C021E001
:1024200030E0023020F4F701859195919C01472D11
:10243000612F802F96D9739422E0E20EF11C38E0D0
:102440007312EDCF1F5F88E0C80ED11C193049F020
:10245000C601880F991FDC01A652BD4F7D01712C6A
:10246000DECF0F5FB8E48B0E911C0430A9F63BDE83
:10247000FE013196DF011D921A95E9F78FEF9FEF6C
:102480009E838D8387E08A8701E912E07F014AE01D
:1024900050E0B801C7010E94CC2E065F1F4F013EDD
:1024A000B2E01B07A1F7B0924102A09240022A9627
:1024B000EDE00C94392E9C01CB01BA01F901329662
:1024C000E4914E2F50E06E17710548F0F9013496F3
:1024D000659175910E94722E80E090E008958FEFD3
:1024E0009FEF0895A4E0B0E0E8E7F2E10C94252E18
:1024F0008B01FC013396F49019821A821B821C8294
:10250000452B31F48FEF9FEF2496E5E00C94412E9C
:1025100044E050E0BE016F5F7F4FCDDF019691F345
:1025200081E090E00F2C02C0880F991F0A94E2F717
:10253000092E000CAA0BBB0B49815A816B817C814F
:1025400084239523A623B72321E0892B8A2B8B2B69
:1025500009F420E0F801208380E090E0D5CF9C01D1
:10256000CA01F9013296E4914E2F50E08E17910581
:1025700050F0F9013496859195910E94722E70DD8C
:1025800080E090E008958FEF9FEF0895A4E0B0E021
:10259000ECECF2E10C94212E7C016B01CA01F701F5
:1025A0003396B49019821A821B821C82892B31F4D3
:1025B0008FEF9FEF2496E9E00C943D2E44E050E02D
:1025C000BE016F5F7F4FC70176DF019689F381E01F
:1025D00090E00B2C02C0880F991F0A94E2F78095B7
:1025E0009095092E000CAA0BBB0B49815A816B8177
:1025F0007C8184239523A623B723F6012081022F13
:10260000017010E00B2C02C0000F111F0A94E2F7BA
:10261000012E000C220B330B802B912BA22BB32B02
:1026200089839A83AB83BC8344E050E0BE016F5F33
:102630007F4FC70194DFBECFA9E0B0E0E2E2F3E153
:102640000C941B2EFE01319689E0DF011D928A95C4
:10265000E9F78DE2E82E81E0F82E8F0196E3C92E8E
:1026600091E0D92E3F01AA24A394B12C3EE3832EFE
:1026700031E0932EF70181917F018F3F09F43EC035
:10268000F894E82FE295EF70F0E021A18F70A5019A
:1026900002C0440F551F8A95E2F7CA01922F982B6A
:1026A00091A392A18095892382A3789400C0E6E348
:1026B000F1E031E0512C21912F3F79F0A22FA2952A
:1026C000AF70A05EB0E08C9190E02F7002C0959545
:1026D00087952A95E2F780FF35C080E0582A330FAE
:1026E0008E169F0641F7F70182918F3F11F00E94ED
:1026F000EB0650EA5A95F1F7D8015C920F5F1F4F35
:10270000CE14DF0409F0B6CF49E050E0B30185E113
:1027100092E00E94652E892BB9F089E0F301A5E1D2
:10272000B2E001900D928A95E1F781E08093D601A5
:102730000E94AE089093D5018093D4012996EFE0D2
:102740000C94372E832FCACF8091D6018115B1F317
:102750000091D4011091D5010E94AE08801B910B0D
:10276000059760F349E050E065E172E087E392E0AD
:102770000E94652E892B49F089E0E5E1F2E0A7E3AC
:10278000B2E001900D928A95E1F71092D601D6CF72
:10279000A0E1B0E0EEECF3E10C941A2EFE013196CC
:1027A00080E1DF011D928A95E9F702E110E091EEE8
:1027B000A92E92E0B92E2FE1422E55245394612C7C
:1027C000712C4F0173016201B1E14B165104610498
:1027D00071041CF080E1C82ED12CA601B501C40102
:1027E0000E949F2EAC0CBD1C0D2C000CEE08FF08A7
:1027F0004C185D086E087F080150104019F760966C
:10280000E0E10C94362E6FEF85E290E00E94AE2E50
:102810006FEF86E290E00E94AE2E6FEF87E290E0CD
:102820000E94AE2E60E088E290E00E94AE2EE1DDD4
:10283000AFDF66E285E290E00E94AE2E66EE86E2B1
:1028400090E00E94AE2E60E487E290E00C94AE2E01
:10285000A2E0B0E0EEE2F4E10C94282E63EE7EEF0D
:1028600080E090E00E94C82E60E082E090E00E944C
:10287000AE2E81E080933D0361E083E090E00E9412
:10288000AE2E198284E18A83CE0101960E94990BB3
:10289000BADF40E050E0BA018FE090E00E94C02E25
:1028A00040E050E0BA0183E190E00E94C02E229601
:1028B000E2E00C94442EEBEFE80FEF3308F070C029
:1028C000F0E0E151F14D0C944F2EC2DF81E008950C
:1028D00080912002807F8093200281E080939F027C
:1028E000F5CF8091400290914102892B79F311D864
:1028F0002FEF84E39CE0215080409040E1F700C03E
:1029000000000E94980990912002892F8E7F90FFED
:1029100081608093200280FDD9CF817F8093200247
:10292000D5CF90912002892F8D7F91FF8260809377
:10293000200281FFCBCF809120028160EFCF909168
:102940002002892F8B7F92FF84608093200282FD7A
:10295000F2CFBCCF90912002892F877F93FF8860B0
:102960008093200283FDE7CFB1CF0E94890C909124
:10297000B103892F97FB87F980588093B103A6CFC5
:1029800081E00E94A3030E94890CA0CF895391E0AB
:1029900001C0990F8A95EAF7892FF3CF8D51F7CFB0
:1029A00080E00895CF93C82F8115B9F18CEF8C0F7B
:1029B000813A08F054C080919F02811529F081303E
:1029C000F1F010929F0208C080913F03823221F4FF
:1029D0008C2F71DF811121C0809110018130F9F0BD
:1029E000EEEAF1E08191C817A1F121E0E43BF207A2
:1029F000C9F78C2F0E944B080E94D70B0EC0809104
:102A00003F03823229F3C932E1F228F4CB3029F0B6
:102A1000C431B9F2E1CFC833F9F6CF91089580916E
:102A2000B10387FFDDCFEC2FE695E695E695F0E064
:102A3000EC54FE4F828190E04C2F477021E030E053
:102A400002C0220F331F4A95E2F782239323892B7A
:102A500081F28C2F0E947F080E94D70BCACF80E2A0
:102A60008C0F883048F4C77081E001C0880FCA9588
:102A7000EAF70E94E104C0CF8BE58C0F833038F475
:102A80002C2F2452330BC9010E94FB07C6CFC85A12
:102A9000CB3118F6EC2FF0E0EE0FFF1FEC58FE4F95
:102AA000808191810E942308B8CFCF93DF93EC01FE
:102AB000805E9109089720F060E37CE0209711F494
:102AC0006BE27CE0CE010E9463038C2F6BDFDF9111
:102AD000CF910895611529F020914203226020933F
:102AE00042039C0130522115304308F49927DDCF71
:102AF000CF92DF92FF920F931F93CF93DF93EC015E
:102B00008B01F42E8091130182FF63C0C0902D03CE
:102B1000D0902E03CC16DD0619F0209709F059C08D
:102B2000809113018B7F80931301C1E081FD10C060
:102B300080912B0390912C039801281B390BC1E045
:102B400080910C0190910D012817390708F4C0E01D
:102B500080911301C0FB81F9809313016C2FC60192
:102B60000E947E0780913F0381FF08C0809113017E
:102B700080618093130182E00E94E70480913F030B
:102B800085FF08C08091130180628093130180E269
:102B90000E94E7046C2FC6019DDFF11431F0809193
:102BA000A40385FF02C086FF28C08091A7039091EF
:102BB000A8030E94290B80912D0390912E039C0164
:102BC00030522115304308F499270E94740CCBD958
:102BD00010C0CE01905281159043B8F4CE019927D0
:102BE0000E94740C80912D0390912E03C817D90771
:102BF00071F310932C0300932B03DF91CF911F915E
:102C00000F91FF90DF90CF900895CE01E9CF1F93F1
:102C1000CF93DF93182FEB01C5DE209739F4812F76
:102C20000E94510CDF91CF911F9108958FE99FE091
:102C30000197F1F700C000002197EFCF6091A90341
:102C40007091AA03893321F06091A7037091A803C2
:102C5000DECFEF92FF920F931F93CF93DF93C62F98
:102C6000D42F122F8115A9F0609336030E94AE086D
:102C70009093D8018093D701C77081E001C0880F7D
:102C8000CA95EAF70E942B0CCDB7DEB7E6E00C94AC
:102C9000402E80913603681331C0E090D701F09048
:102CA000D8010E94AE088E199F09883C910530F525
:102CB00000E20D0FCD17A9F0C770FF24F3948F2DFC
:102CC00001C0880FCA95EAF70E94390C083048F411
:102CD0008D2F877001C0FF0C8A95EAF78F2D0E9417
:102CE0002B0C812FABDF083078F6D77081E001C064
:102CF000880FDA95EAF70E94390CC6CFC77081E0D9
:102D000001C0880FCA95EAF7F6CFA0E0B0E0EBE883
:102D1000F6E10C94212EEC0188818115E1F08130DF
:102D200009F040C08981813021F48A81239686DFB1
:102D3000F3CF823021F48A81239634DEEDCF8330C5
:102D400029F48A8123960E94510CE6CF843041F009
:102D500022968111E1CFCDB7DEB7E9E00C943D2E8C
:102D60008A81239620E030E09AE0682F6053770B49
:102D7000AB016A30710560F02115310551F3EFE9BF
:102D8000FFE03197F1F700C0000021503109F4CF86
:102D9000929FB001939F700D11249A01260F371F47
:102DA0008991E3CFE82FF0E0E155FE4FB490282F52
:102DB00026952695269530E0F901E156FE4FE490E0
:102DC0008770F12C082E02C0F594E7940A94E2F77C
:102DD000E0FAEE24FF24E0F8F901E157FE4FC49039
:102DE000D12C082E02C0D594C7940A94E2F7C0FAF9
:102DF000CC24DD24C0F8F901E158FE4F049110E025
:102E000002C0159507958A95E2F701701127E11424
:102E1000F10411F081EEC6DDC114D10411F086EE8B
:102E2000C1DD60E070E08B2DF2DEC114D10419F039
:102E300086EE0E94510CE114F10419F081EE0E941B
:102E4000510C0115110511F08CE2F8DE219664CFCA
:102E5000AEE0B0E0EEE2F7E10C94182E7C01DC016C
:102E600014968C91811511F40C94912160E0C701A6
:102E700011DA9C01F7018681803170F44091490399
:102E800090914803491333C090918703911521F025
:102E900090918803903158F1D70115969C9191112A
:102EA00010C02115B0E53B0708F088C02115E0E20D
:102EB0003E0708F098C0283E310590F4203E3105C9
:102EC000B0F43093A1022093A002D70112968D9105
:102ED0009C9190934703809346031092140107C07E
:102EE000C9019A9581159F4160F72111EACF61E0F0
:102EF000C701D0D98C01F7014581411511F40C941B
:102F0000582197578038910510F00C9474210031A6
:102F100010F00C9480216EE171E080E090E0C0D967
:102F200081110C948021812C912C540101115DC0E0
:102F300004E0AE014F5F5F4F1A01D101E02F1D92F7
:102F4000EA95E9F724013501FFEF4F1A5F0A6F0A8E
:102F50007F0AC501B401A4D98983811511F40C94A9
:102F60008021813009F0D1C0A50194012E5F3F4F2F
:102F70004F4F5F4F2F83388749875A87C301B2016C
:102F80008FD9182F8A83811511F40C9480218FEF2B
:102F9000810F833008F043C06F81788589859A85D9
:102FA0007FD98B83811511F0C101AFDE240135017A
:102FB00033E0430E511C611C711C6EC0203E42E583
:102FC000340760F4203852E5350708F090CFC90186
:102FD00080529245809708F074CF89CFC9018757F6
:102FE0009C470297F8CF8031F6CFFFE18F16F1E0D2
:102FF0009F06A104B10411F40C948021C501B40111
:103000004FD92FEF821A920AA20AB20A8111EDCF8C
:1030100001508CCF4F80588469847A843DC08BEFF7
:10302000810F8330E0F52401350143E0440E511C4B
:10303000611C711C6F81788589859A8531D98B8354
:10304000811551F1C301B2012BD98C838115E9F0AF
:10305000CB80DC8051E0C5165FEFD50610F0DC2C8C
:10306000CC24163079F0173049F0C6010E94C826EA
:103070008091A7039091A8030E94290BC6010E948A
:10308000E72603C0C6010E94C8262401350154E08A
:10309000450E511C611C711C530142014ECF14306E
:1030A00009F0B8CF6F81788589859A85F9D8182F6E
:1030B0002401350184E0480E511C611C711CC501BE
:1030C000B4016D5F7F4F8F4F9F4FEAD8111511F4F8
:1030D0000C948021811511F40C9480218150990B5E
:1030E0004FEF489F9001499F300D1124A12FA1500F
:1030F000BB0B2A0F3B1F2150310970F2EFE9FFE0B3
:103100003197F1F700C00000F6CFC101FEDDC4CF5A
:1031100010923F030E94EF040E94AE0888579C4E15
:103120009093A4028093A30281E08093A2020C9466
:103130008021023B82E5180709F03FC025EE30E010
:103140002770332781E090E001C0880F2A95EAF7C5
:103150002091A5023091A2023115F1F04115B1F094
:10316000282B2093A5020C948021D70116968C91D0
:10317000803118F5812F99278F7199278230910519
:1031800011F04297D9CF21EE30E0DACF809582233B
:103190008093A5020C948021322F3823311569F0D9
:1031A000982F909592239093A5020E94E704F7012F
:1031B0008581811511F40C9480218091A2028115E2
:1031C00009F475C0C0903F03D0903B030E94AE0845
:1031D00088579C4E9093A4028093A302D701159622
:1031E0008C91811509F463C08D2D8C298D79811105
:1031F00086C00115B0E51B07B0F50115E0E41E0718
:1032000008F084C0063E110509F451C0C80190526F
:1032100081159042E8F5D70116968C91803108F41B
:1032200068C0C80199272091130120FF79C02DEFB4
:103230002095309142032323209342038D32910540
:1032400071F008F07EC08832910508F06BC08E31B5
:10325000910508F069C004974A9708F050C082E0D1
:103260008093420361C0003EB2E51B07C0F4003CFE
:10327000E2E51E07E0F4003AF2E51F0758F40036D5
:1032800022E51207A0F4C80192558034910578F028
:10329000C801C9CF043B32E5130749F0F9CF09371C
:1032A0004CE7140710F507375CE7150788F3F701BB
:1032B0003580311409F44FC00E35FCE71F0709F4BF
:1032C00046C00F352CE7120749F00D353CE71307D0
:1032D00009F041C0809112018115C9F110921201CB
:1032E00080E00E94D60F0C9480210B378CE71807E2
:1032F000D4CF812F8F718431D1F2863171F00E9449
:10330000480C8091A5020E94E104D1CFD701169606
:103310008C91803108F085CFCACF86EE92E183CFC1
:103320002FEF86CF8A9759F78091A502811531F04A
:103330008091420392E08927809342030E94D70B39
:10334000B6CF8C34910581F38D329240ECCF81E081
:1033500080931201D5C780911201811150C08091D4
:10336000A40380FF27C20E94AE085C01D701159616
:103370008C91811509F42FC28091130182FF05C041
:1033800040E0B50180E090E0B3DB0431BCE71B070F
:1033900009F41DC20531ECE71E0709F4B6C103317B
:1033A000FCE71F0709F4F8C1C8019052811590434A
:1033B00008F0B5C110922E0310922D03D701159677
:1033C0009C91911509F464C310923603980130570B
:1033D0002332310508F05CC384E090E00E949A2E0D
:1033E0009093B2038093B103F801E150F047E232C9
:1033F000F10508F097C2E25DF04D0C944F2E3801B4
:1034000040EE641A710850903C0380913F03582AA3
:1034100080913B03582A58E06516710408F05EC09D
:1034200098012770332781E090E001C0880F2A952A
:10343000EAF7311409F44FC0582AD7018D919C91B5
:103440000E94F40321E030E0F90102C0EE0FFF1FFB
:103450008A95E2F7FC87EB872091210330912203C4
:1034600038872F834091290350912A035E874D8727
:1034700058EAC52E52E0D52EA12CB12C511005C012
:10348000D60112968C9181111BC0F601838190E0C8
:103490002B853C8582239323892B91F08085982F5F
:1034A0009770911101C087E038E06316710408F04D
:1034B0005AC0311409F453C086958170811158C0E7
:1034C0009FEFA91AB90AAFE0CA0ED11CB8E0AB163B
:1034D000B104A1F61CC080955822AFCF31102CC08A
:1034E0008091290390912A030817190781F41092FB
:1034F0002A0310922903109225031092260310929A
:103500002703109228031092240310922303809122
:10351000210390912203009709F421CFE8E06E1671
:10352000710408F0DEC0652D0E94A407811117CF39
:1035300081E00E94D60F13CF10932A030093290332
:103540000E944B0960932503709326038093270301
:103550009093280310922403109223036ECF82FBD2
:10356000882780F9ABCF311409F4AACF80FFA8CF08
:10357000D6018D909C900815190519F4311409F4A1
:103580009FCFEF81F885EC15FD0509F499CFD601A1
:103590001D96ED91FC91309721F08081811509F401
:1035A0008FCF652DC6010E94A407811509F488CF2D
:1035B00081E00815190509F080E0482E43208114A8
:1035C000910441F0411006C0ED85FE858E169F06E0
:1035D00009F076CF80E00E94D60FD0922203C092ED
:1035E000210381E0809320038FE08A9DF0018B9D71
:1035F000F00D1124E855FD4F85818093A7024110FD
:103600000EC08114910459F0808191819C01245055
:103610003109213A310508F049C00E947F088FE046
:103620008A9DF0018B9DF00D1124E855FD4FC68059
:10363000D780C6019A9581159F4110F420EED222C1
:1036400099249394C60101978F339E4708F0912CDB
:103650008FE08A9DD0018B9DB00D1124A855BD4FE0
:103660001996ED91FC911A97309731F01B966D9158
:103670007C9181E0099598229114A9F08FE08A9DB0
:10368000F0018B9DF00D1124E855FD4F8681978147
:103690000E9439038093A602C60148E064167104B3
:1036A00040F40E9457090E94D70B0AC00E94510C97
:1036B000B6CF0497813A910548F48C2D0E944B08AF
:1036C000411409F44CCE0E94D70B1AC60E94D70BA6
:1036D0008FE39CE90197F1F700C000008C2D62D9BF
:1036E000EFCFDC012D913C910217130731F431101B
:1036F00007C01092200380E01CCF311409F42FCEB4
:10370000FC01808585FD2BCEF6CF90911301892F8A
:103710008E7F90FF8160809313010E94B30F809190
:10372000130180FF47C00832110508F06AC00E314E
:10373000110508F077C0C80104974A9790F5809169
:10374000A40384FD2EC0D70115968C91811509F430
:10375000C8C090913F0380913B03D82ED92A2D2DCC
:103760002D7F211509F463C010922E0310922D03B2
:103770002091A40321FD5BC060E0C8010E947E0788
:1037800060E0C801A7D980913B038D7F0E94380972
:1037900082E00E94C604B4C58091130181608093C9
:1037A0001301D70115968C91811521F010922E03EB
:1037B00010922D03F7018581F801E851FC47E730AD
:1037C000F10508F0FBCDE05BF04D0C944F2E80919D
:1037D00013018E7FA0CF809113018F7E013E1105D2
:1037E00031F0053E110531F4809113018F7D8093F6
:1037F000130195CFC80190528115904308F08FCFE7
:10380000DDCD0933110558F40D32110518F40B32D2
:10381000110539F68091A40382FDC3CF94CF0436FD
:103820001105F7CF8091A40383FDBBCF8CCF27E098
:10383000F701AFE2B3E001900D922A95E1F7109203
:1038400032031092310380902D0390902E030815BF
:10385000190589F52091A40325FF2DC0309113018E
:1038600031FBCC24C0F831FF02C026FF24C02091D8
:103870002B0330912C03F501E21BF30BE83CF1051F
:10388000D0F491FF08C080911301806180931301EF
:1038900082E00E94E70480913F0385FF08C0809189
:1038A000130180628093130180E20E94E7046C2D73
:1038B000C40110D925C58D7F0E94380910932E03AD
:1038C00000932D03B0922C03A0922B038D2D8270B8
:1038D000846090911301997FD82ED92AD092130138
:1038E00057CF40E0B501C80103D90AC526E241EE31
:1038F00061EEAFD905C527E245EE65EEFACF26E2C7
:1039000041EE60EEF6CF27E245EE64EEF2CF26E21E
:1039100041EE62EEEECF27E245EE66EEEACF28E218
:1039200041E0EBCF8091B10381608093B10381EBE3
:1039300093E00E94990B0E94890CE2C48091B2032B
:1039400088608093B203F3CF8091B1038260EDCFA2
:103950008091B1038460E9CF8091B1038860E5CFA5
:103960008091B2038160EDCF8091B2038260E9CF94
:103970008091B1038061D9CF8091B1038062D5CFAE
:103980008091B1038064D1CF0E94890C8091B103F2
:103990008068CBCF8091B1038C60C7CF8091B20398
:1039A0008360CFCF8091B1038E7FBFCF8091B20370
:1039B000877FC7CF8091B1038D7FB7CF8091B1034F
:1039C0008B7FB3CF8091B103877FAFCF8091B2035C
:1039D0008E7FB7CF8091B2038D7FB3CF8091B1033B
:1039E0008F7EA3CF8091B1038F7D9FCF8091B10354
:1039F0008F7B9BCF0E94890C8091B1038F7795CFED
:103A00008091B103837F91CF8091B2038C7F99CF56
:103A10008091B103992782FF939590FB82F990FBE7
:103A200083F983CF8091B203982F909590FB80F912
:103A300090FB81F986CF9091B103892F8F7B96FF00
:103A4000806473CF0E94890C9091B103892F97FBFA
:103A500087F980586ACF61E08EE090E00E94AE2E38
:103A600066CF60E0F9CF9091B103892F8F7E94FFEC
:103A700080615BCF9091B103892F8E7F90FF816031
:103A800054CF9091B203892F877F93FF886059CFDD
:103A90000631BCE71B07C1F580913F033091A303BA
:103AA00030FF04C0282F2474211122C0282F2A7A25
:103AB00031FF04C0482F4171411120E032FF04C0A2
:103AC000482F4878411120E033FF03C082728111F2
:103AD00020E0911579F081E0211101C080E0809310
:103AE000370385E3211101C089E20E944B08EBCD29
:103AF00020E0DECF80913703811521F085E30E941D
:103B00007F08E1CD89E2FBCF0737ECE71E07F9F02C
:103B10000837FCE71F0731F19801205E324520325B
:103B2000310528F5911123C00F7181E090E09C01CF
:103B300002C0220F331F0A95E2F78901622F83E04A
:103B400090E00E94AE2E802F0E94A303D9C381E093
:103B5000911551F00E94A90343E062E081E00E94C8
:103B60002704CEC382E0F4CF0E94B303F5CF409187
:103B7000380380913E03282F30E02095309570E087
:103B800024233723232B19F04823409338030B3782
:103B90003CE7130741F4911509F4B2C30E946C038A
:103BA0000E94C507ADC3003442E5140708F055C0B4
:103BB000003252E5150708F057C0011580E51807D7
:103BC00050F50115A0E41A0708F064C0911509F436
:103BD00079C00A35FCE71F0709F403C108F0E8C003
:103BE00001303CE7130709F4FAC003304CE714072F
:103BF00009F4EFC001151C4709F064C00E94890C4C
:103C0000AFEFB4E3ECE0A150B040E040E1F700C01A
:103C100000000E9498099801305521153240B0F6F5
:103C2000980145E0369527954A95E1F7822F8F70E8
:103C30002091380330E041E050E0082E02C0440FEC
:103C4000551F0A94E2F724233523232B09F4BECF12
:103C50009111A6CF10923F0336CD9801205C3245DA
:103C60002032310508F0B2CF802F8F7120913803B8
:103C700030E041E050E0082E02C0440F551F0A9486
:103C8000E2F724233523232B09F4A0CF911509F45F
:103C900037C386CFF7018681803108F097CF911125
:103CA00011C0212F2F7081E090E002C0880F991F72
:103CB0002A95E2F72091380330E082239323892B61
:103CC00009F01EC3F7018581C080D180811509F4F8
:103CD0008CC0C6010E94EC10182F682FC6010E94EC
:103CE000C103B601812F0E94D1100E94ED05082F5B
:103CF000D92E86E0F701DE01119601900D928A958A
:103D0000E1F7D7011596BC9015971696CC90C29402
:103D10009FE0C922809143038770811501F19B2C9C
:103D2000B114F1F08D2D807F803461F080E2800F3E
:103D30008830A8F08D2D807E803221F4023078F01A
:103D4000C11469F08091B20382FF09C082E00E9431
:103D5000C604809143038770992493948111912C18
:103D6000AD2CA2948FE0A822B8E0AB1609F46DC187
:103D7000E9E0AE1608F074C0F4E0AF16D8F51D2DDA
:103D80001F7022E0A21608F47EC08D2D807F803245
:103D900011F01295107F011509F4ACC0013009F43F
:103DA00016C1B11409F422C1C11409F4BDC07FC009
:103DB0000B358CE71807B9F08091B203002482FF1D
:103DC0000394802D0C351C4709F07CCF0E94A00B7A
:103DD00079CF6FEF7FEF80E090E00E94C82E0E94C5
:103DE000A70C81E0F3CF80E0F1CFC6010E94F4037D
:103DF000182F77CF34E0A31609F40AC1AA2DA850D2
:103E0000BB0B149718F40E94EC07912C802F9D2D6A
:103E10000E947F03811541F0B11409F41EC2C11440
:103E200009F412C21092B5039114A9F080914303D2
:103E300080FD11C0D70115961C92869586958695B2
:103E40000E94A903C70104D88091430386958695F3
:103E500086950E94B30360E0C7010E944A1161C2C7
:103E600049E0A41609F461C186E08A0D8F708230A2
:103E700028F6023F09F069C18D2D8F71B11062C122
:103E80000E94A903BBCF50E1D51610F01295107F08
:103E9000B114B9F0111559F080E2800F883010F09C
:103EA000011109C0812F0E94E1040E94D70B802FCD
:103EB0000E94D214A3CF80914203812B80934203AE
:103EC000F4CF802F0E94510C111509F497CF80E296
:103ED000800F883010F0011104C0812F0E94E70488
:103EE00006C01095809142038123809342030E9473
:103EF000D70B84CF8091B20382FD12C0B11449F078
:103F0000111529F0812F0E94E1040E94D70B80E057
:103F1000CFCF80E00E94510C111509F46FCFDDCF97
:103F2000B11491F1C11004C0812F0E942B0C66CFF7
:103F3000B1E0CB1211C080903B03812F882118176C
:103F400009F45CCF0E94AE0890933A038093390342
:103F5000812A80923B0352CF8091A503823008F4DE
:103F60004DCFC8124BCF812F0E942B0C812F0E9466
:103F7000230980913C03912F9823191709F43ECF10
:103F8000812B80933C033ACFC11012C0812F0E9435
:103F9000390C812F0E94230980913C03912F982393
:103FA000911509F42BCF1095182310933C0326CFBD
:103FB0008091A503823008F421CFE1E0CE121ECF1C
:103FC00080913F038123811509F418CFDFCF8091C1
:103FD000AB03B11421F08C1508F410CFA5CFC8168F
:103FE00008F00CCF812F0E94390C08CFC114D1F3F7
:103FF0008091A9039091AA03093321F08091A7032E
:104000009091A8030E94290B802F0E94510CF6CE9C
:104010008D2D869586958370811569F0813009F024
:10402000EDCE802F9D2D9370B11002C080E090E006
:104030000E942308E3CE802F9D2D9370B11002C003
:1040400080E090E00E94FB07D9CE8D2D8370811116
:1040500033C0B110D3CE402F429546954770440FE0
:10406000440F802F8F70042E01C0880F0A94EAF746
:10407000202F207104FF07C02FE030E001C0220F85
:104080004A95EAF720953D2D3695369533703230B6
:1040900071F0333051F040913D03313029F0822BE3
:1040A00084230E94A303AACE842B822BFACF822BD7
:1040B00090913D038927F5CFB11459F1D0FE9ECEE2
:1040C000402F429546954770440F440F802F8F70C4
:1040D000042E01C0880F0A94EAF7202F207104FFF4
:1040E00007C02FE030E001C0220F4A95EAF7209583
:1040F0003D2D369536953370323091F0333071F076
:1041000040913E03313049F0822B84230E94A60364
:1041100075CE823008F472CED3CF842B822BF6CFAB
:10412000822B90913E038927F1CF1D2D1F70B11472
:1041300029F0812F0E94A903802FF7CE802F0E94A3
:10414000390C812F0E94B30359CE60F4003FB9F0BF
:10415000013F81F0B11409F472C0C110A8CE8D2DB9
:104160008F718ECE033FF9F0043FA1F78091B20327
:1041700082FD25C08D2D8F71B11421F381CE8091E8
:10418000AB03B11461F0C81608F038CE2D2D2F7195
:1041900081E090E001C0880F2A95EAF7C2CF8C1524
:1041A00008F42CCEF3CF80E0B11409F4AFCF81E056
:1041B0009D2D9F7101C0880F9A95EAF7A7CF809136
:1041C000A503823048F1B114C9F090914303977070
:1041D000943059F410924303109245031092440313
:1041E0008D2D8F710E94B3030ECE63E0C81608F0C8
:1041F0000ACE8D2D8F710E940F0905CEC81640F092
:1042000010924303109245031092440364E0F1CFEF
:1042100081E00E94C604F7CDB11431F063E08D2D2A
:104220008F710E940F09EACD81E00E94C604F2E07E
:10423000CF1608F4E3CD82E00E94C604DFCDC110A2
:10424000D7CE8D2D8F717ECF809141038093400317
:1042500080913F0380934103E7CD40E060E0898196
:104260009A810E942E119C0110913F03C11429F0E4
:104270001092B50310934103D7CD8091B303909171
:10428000B40328173907B1F78091A60382FFF0CF56
:104290008091B503811561F3809140030E942B0C3E
:1042A000802F0E941E16809140030E94390CE0CF9F
:1042B00083379C4729F1023A22E5120711F40C9446
:1042C000C31810F00C949918C801905281159042AF
:1042D00010F40C94B518013E110511F40C94C31898
:1042E000053E11050C949C180337ECE71E0719F7DF
:1042F0008091A202811511F40C9488180E94480C38
:10430000809143038770811561F0D70115968C91D8
:10431000811539F08091B20382FF03C082E00E94D0
:10432000C6042E96E2E10C94342E809188038031ED
:1043300078F480918703811559F0E0914903209129
:104340004803309183034091820357E02E1301C04C
:1043500008956E2F70E05E9FF0011124DF01A65BCF
:10436000BC4F14968C911497811559F111968C912C
:104370001197831326C08C91841323C015968C91BA
:10438000159781111EC012968D919C91A091840366
:10439000B09185038A1B9B0B883C910590F480911A
:1043A00088038F70806180938803E05BFC4F80817D
:1043B0008F708061808382E893E00E9428170C94BC
:1043C000BC04FB013196E770C1CFCF92DF92FF9220
:1043D0000F931F93CF93DF93182F092F87E0F82EA9
:1043E000C091490380914803C81799F1FC9EE001F0
:1043F0001124CE01865B9C4F6C01FC0185818115E7
:1044000089F0C6010E942311811561F0FE01E05B75
:10441000FC4F20812F7020612083F60180819181E3
:104420000E94BC0CC6010E9428172091490330E06D
:104430002F5F3F4F2770332720934903C65BDC4F24
:1044400089818013CDCF88818113CACF8D81811559
:1044500039F2DF91CF911F910F91FF90DF90CF90B4
:104460000895EF92FF921F93CF93DF93EC01209179
:104470001401211541F010E0812FDF91CF911F91A0
:10448000FF90EF900895EA80FB80E61AF70A24EF88
:10449000E21621E0F20678F760E0CE010E944A11B0
:1044A0009C0130522115304330F70E94870481155A
:1044B00011F38091A0029091A1020E948704182F0D
:1044C0008115C9F28091AF039091B003853F21E03F
:1044D000920710F084EF91E0E816F90660F68E81FD
:1044E0008F7080618E83888199810E94BC0C0E94AC
:1044F0004604CE010E942817BFCFADE0B0E0E3E84C
:10450000F2E20C941A2E8C0186E0F801DE01189676
:1045100001900D928A95E1F7D8016C9011965C900C
:1045200011971296AD90BC9013971496EC90149737
:104530001596FC90F1100CC050918302252F30E0AD
:10454000E0E08E2F0E2E000C990B821793073CF1A2
:1045500052E8C52E53E0D52E80918603811151C0BB
:10456000E114D1F0F11409F402C3C8010E9423112F
:10457000811509F4FCC26091460370914703C8019C
:1045800070DF811109C087E0F801A2E8B3E0019073
:104590000D928A95E1F7C9DEFF24F39486C0880F57
:1045A000991F8D589D4FDC0111964C911197451123
:1045B00003C08C91681611F0EF5FC3CFEF3F41F25B
:1045C000D80116968C9116978F70806116968C93F1
:1045D000E517A0F4AFEFA50FA0938302EA1770F4DC
:1045E000F0E0EE0FFF1FED58FD4FB0E0AA0FBB1F2C
:1045F000AD58BD4F8D919C91918380830E9446045C
:10460000A7CF60E082E893E00E944A119C0170907D
:10461000870380918403909185034501881A990A44
:10462000711409F451C2B8EC8B16910408F00AC257
:10463000E11409F4B1CF80918303F8019181E090F6
:104640008803F0E1EF1608F0C6C1981350C09091AE
:104650008203D8018C9198134AC0F11048C08E2D66
:104660008F7080618093880382E893E00E9428170E
:1046700080918803F8018683F0908403E09085039D
:1046800047E0D42E0091490380914803081751F068
:10469000D09E80011124065B1C4FD80115968C9189
:1046A000811108C00E94BC04F12C8F2D2D96E0E1F1
:1046B0000C94362EF801B280C380C8010E942311E9
:1046C00081110EC0C8010E9428178091490390E013
:1046D00001968770992780934903FB2CEC2CD2CF4D
:1046E0006F2D7E2DC801BDDE8111EFCFDBCF3052A3
:1046F0002115304308F084C0F11005C140E0652D5C
:10470000862D0E940A0B81114FC040E0652D862D39
:104710000E940A0BF82E811509F429C18091A60385
:1047200080FFC2CF82E893E00E94281760E082E811
:1047300093E00E944A118C01F09049037F2C98E08D
:10474000E92E22E8822E23E0922E37E0432E80913C
:1047500048037816A1F0A72CB12C479CC001112466
:10476000FC01E65BFC4F6F0160E0CF010E944A1143
:10477000582E692ED60115968C91811197C0B8E0FC
:10478000EB1618F417E0EF10ACC0888599851DDE94
:104790000E9446040E94BC0487E0E2E8F3E0DF01E7
:1047A0001D928A95E9F780CF60E0C8010E944A1106
:1047B0008091A60383FFA9CFB80182E893E00E940D
:1047C00053048111A2CF809188038F708061809300
:1047D000880380918203909183030E94BC0C82E83D
:1047E00093E00E942817E2E8F3E087E0DF011D92E2
:1047F0008A95E9F788859985E8DD0E94460452CFBD
:10480000F11409F482CF809188038160809388033A
:104810008091A60381FF48CF82E893E00E94281789
:104820000091490380914803081709F4CCC0E02E99
:10483000F12CB7E00B9FC0011124FC01E65BFC4F9B
:104840006F01CF010E942311811509F4BCC087E0DC
:10485000F601A2E8B3E001900D928A95E1F7C70155
:10486000019687709927082F809349030E94BC0402
:1048700087E0F82E80914803801709F413CFF09E4B
:1048800080011124065B1C4FC8010E942311811175
:1048900009CFC8010E9428178091490390E0019632
:1048A00087709927082F80934903E4CF1052011590
:1048B000E0E31E0708F063CF8091A60383FD0AC0E2
:1048C000E72CC5010196F82FF7707F2E052D162DC8
:1048D00046013DCFB601C4010E945304811589F3FE
:1048E000EFCF1F9DC0011124865B9C4F0E942817AB
:1048F0002091490330E02F5F3F4F27703327F22E7E
:104900002093490340CF809188038160809388037E
:1049100060E0C8010E944A118091A60383FF78CF0E
:10492000B80182E893E00E945304811171CFF090A6
:104930008803E894F0F8F0928803C8010E942311DC
:104940008111B2CE8F2D8F7080618093880380910A
:104950008203909183030E94BC0C0E94460482E86B
:1049600093E00E942817E2E8F3E087E018CF8885FB
:1049700099850E941611292F22952F70903450F49A
:104980009F70223080F0911599F0F8019681903156
:1049900078F48BCE2A5F2F70223078F0C8010E9405
:1049A0002817F72C82CE911519F0811509F47DCEC8
:1049B000805E883008F479CEF1CF803F08F475CE60
:1049C000815F8330F7CF87E0E2E8F3E0DF011D92FB
:1049D0008A95E9F74DCF981315C090918203F8019D
:1049E000808198130FC0F1100DC0E682C8010E94AB
:1049F000281787E0F801A2E8B3E001900D928A95AC
:104A0000E1F7CACDC8010E942311811509F4AFC096
:104A1000F11409F4ACC080918803803208F4B3CD5E
:104A200080918203909183039A838983BC82AB82B5
:104A3000809186038D831E82EF82CE0101960E94B3
:104A40002817A1CD90908803F0E19F1638F482E8F2
:104A500093E00E94281787E0D601A2CEE11409F462
:104A60009BCD90918303F8018181981311C090919F
:104A70008203808198130CC0F1100AC09682C8018D
:104A80000E94281787E0D6011D928A95E9F784CD08
:104A9000C8010E942311811509F469C0F11409F4B9
:104AA00066C080918803803208F46DCD80918203C6
:104AB000909183039A838983BC82AB828091860321
:104AC0008D831E829F82B9CFB8EC8B16910408F0BB
:104AD00052C0E11409F460CDF11409F448C090917A
:104AE0008303F801818198132AC090918203808109
:104AF000981325C060E082E893E00E944A118091FB
:104B0000AD039091AE038816990608F072CF80919C
:104B1000880380FD6ECF803108F46BCFD8011696E4
:104B20008C931697982F907F903F09F45FCF982F22
:104B3000907F905F8F70892B16968C9357CFC8010A
:104B40000E942311811571F0609146037091470313
:104B5000C80187DC811509F416CD87E0E2E8F3E0AF
:104B6000DF0192CF80918803816080938803C80120
:104B70000E94281711CD87E0F60111928A95E9F776
:104B800093CDABE1B0E0E7ECF5E20C94242E4E8B34
:104B90005F8B688F798F082F8A8F192F9B8FF82E44
:104BA000E92E811509F4A0C040E0692F8E899F8904
:104BB0000E942E119C01111549F01092B50390939B
:104BC000B4038093B303109242030AC08091B303ED
:104BD0009091B4038217930719F481E08093B50391
:104BE0001D8A86E0FE017696DE011F9601900D92E9
:104BF0008A95E1F78091B20382FF21C080918B03F7
:104C000090918C03892BD9F00E94AE082091440327
:104C100030914503821B930B20918B0330918C03C1
:104C20008217930738F08091430382FD03C082E02E
:104C30000E94C6040E94BA0881110E94EF04F11478
:104C400061F00B8B1C8B61E0CE010F960E944A1124
:104C500061E0CE010F960E944A110B8B1C8B87E0FE
:104C6000FE013F96DE01189601900D928A95E1F7BC
:104C7000CE01089642DC811110C02091480330918A
:104C8000490387E0FE013896DE01119601900D92EE
:104C90008A95E1F78C8581112BC017E0809149033B
:104CA00090914803891741F0189FC0011124865B39
:104CB0009C4F23DC811143C08C85811112C08091EF
:104CC000140181110EC08A859B8520914603309185
:104CD0004703821B930B8F3F9F4318F081E0809323
:104CE00014016B96E6E0CCC7911509F479CF6BCF30
:104CF000822F90E00196877099273817190671F472
:104D00000E94890C109248031092490387E0E2E860
:104D1000F3E0DF011D928A95E9F7BFCF97E0929FFC
:104D2000D0011124A65BBC4FFE01319601900D927B
:104D30009A95E1F7809348030E94BC04AECF80911E
:104D4000490390E001968770992780934903A6CF85
:104D5000A6E0B0E0EDEAF6E279C70E94AE088C0169
:104D600080914702909148028017910771F0198253
:104D70001A820E94AE08BC0149815A8180E090E00D
:104D800000DF10934802009347022696E4E07AC7BA
:104D9000A6E0B0E0EDECF6E25BC7909344028093AE
:104DA0004302811520E2920728F40E9455152696A9
:104DB000E2E06AC780EF89838A830E94AE0881603F
:104DC000BC0149815A8181E091E0DBDEF0CFA6E0B1
:104DD000B0E0ECEEF6E23CC79093440280934302CD
:104DE000811520E2920728F40E94740C2696E2E0D6
:104DF0004BC780EF89838A830E94AE088160BC0123
:104E000049815A8181E090E0BCDEF0CFCDB7DEB7BA
:104E1000AC970FB6F894DEBF0FBECDBF85B78068E4
:104E200085BF85B7806885BF84B7877F84BF0FB68D
:104E3000F894A8958091600088618093600010923A
:104E400060000FBE80E890E00FB6F8948093610098
:104E5000909361000FBE81E08093110189EE96E08E
:104E60009093AB018093AA010E947A110E944D1089
:104E70000E94530A0E94B00A8091E20084608093ED
:104E8000E200789480914202811599F08091E900C6
:104E90001091EC008F70179511271795182B109211
:104EA000E9008091E80083FD0E94F00C1F701093D0
:104EB000E90082E084BD93E095BD9AEF97BD8093B1
:104EC0006E000E946111811102C00E9403140DE264
:104ED00011E056E3E52E51E0F52ED8018D918D01BC
:104EE0008F3F11F00E94EB06E016F106B1F706E3E2
:104EF00011E0F80181918F018F3F11F00E94EB06C4
:104F0000F1E00E331F07A9F789E0E7E3F2E0DF01E4
:104F1000282F1D922A95E9F7E5E1F2E0DF011D92C5
:104F20008A95E9F780E090E005D7833E9E4F21F413
:104F30000E946111811102C00E94281482E090E059
:104F4000F1D68093200284E090E0F4D69093B203EF
:104F50008093B1030E941C13EFEFF6E721E0E150CC
:104F6000F0402040E1F700C000000E941C13809137
:104F7000370280FF07C06FEF7FEF80E090E008D737
:104F80000E94980983E090E0CDD60E94A30380E0C0
:104F900091E090936A02809369028091420210E44A
:104FA000853009F47BC00E941C1301E212E047E344
:104FB000E42E42E0F42ED701F80191918D912AE27E
:104FC00032E02E173F0709F473C09817B1F3D12CC4
:104FD000D701CD907D01F80191908F019C1421F1B2
:104FE0009C24B12CAA24A394892D8A218115A9F08F
:104FF000B982DA820E94AE089C838B83F1E0FD8344
:1050000091E08C2D8A21811101C090E09E8349811D
:105010005A816B817C818D81B4DDB394AA0C28E028
:10502000B212E2CFF801C292D39439E0D312D0CFBA
:105030000E944B0940C080914202843019F11092C5
:105040001E0288E190E00FB6F894A8958093600066
:105050000FBE1093600083B7817F846083BF83B7E6
:10506000816083BF7894889583B78E7F83BF0FB6A6
:10507000F894A895809160008861809360001092F8
:1050800060000FBE0E941C13E7E3F2E081918111E2
:1050900006C4A0E4B2E0AE17BF07C1F78091420298
:1050A000853009F4C8CF0E94890C0E94EC077BCFA1
:1050B00098138DCF4DDE0091230310912403011529
:1050C000110591F1C0902E02D0902F02E090300295
:1050D000F09031020E944B096C197D098E099F09DD
:1050E000C0902A02D0902B02E0902C02F0902D026A
:1050F0006C157D058E059F05B8F0C8010E945515F9
:10510000109224031092230310922E0210922F0269
:10511000109230021092310210922A0210922B0249
:1051200010922C0210922D028091A40380FF1CC0CB
:105130008091130182FF18C00E94AE08BC018091CB
:105140002B0390912C039B01281B390B80910C01A0
:1051500090910D012817390738F041E080912D0317
:1051600090912E030E9478158091A202811569F01A
:105170000E94AE082091A3023091A402821B930BDF
:105180008F3F9F4710F40E94480C0E94EC079091BB
:105190003202891721F0809332020E944B098091DC
:1051A0004202843009F0F9CE83E08093E9008091D7
:1051B000E80082FFF2CE8091E80090E085FF0BC00E
:1051C0000E94220A30E2E32EF12C8E010F5F1F4F66
:1051D000811561F191E08091E8008B778093E80080
:1051E000911509F4DACE0091450210914602E98149
:1051F0000115110549F1EE3F09F047C08A8183305E
:1052000020F08550833008F040C0EA81EE3008F08D
:105210003CC0F0E0E95AF04D42C58091F100D80160
:105220008D938D01B1E0EB1AF108A1F28091E800B5
:1052300085FDF3CF8091E8008B778093E8000E9492
:10524000220A811599F3C6CFE43148F4E11549F0FB
:10525000E150E33130F4F0E0EB59F04D20C5EE3F82
:10526000A1F28FEF48C31A8289E08B830EC08A8136
:10527000823081F08330B1F0813099F70E944B0980
:1052800014D56B837C838D839E83CE0101960E940F
:10529000720A83CE88E290E045D51B821C821D8273
:1052A0008E83F3CF8091400290914102892B69F364
:1052B00089E0E7E3F2E0DE01139601900D928A9512
:1052C000E1F7E3CF8A81823061F66B817C818D8149
:1052D0009E81EBD488E290E041D5D7CF4C816B81A1
:1052E0008A810E94A3109827892798279E838D83FF
:1052F000CCCF2D813E813227232732274C816B81F1
:105300008A810E94B10BC1CF0E94F911BECF80E10A
:105310008A83BBCF81E08A838FE1A7CF0C810D31D7
:1053200008F0B3CF8A809B80982489249824A12CEC
:10533000B12CFE0131967F010E0F1F2F111DE016BB
:10534000F10609F4A2CF80E0FFE18F16F1E09F069D
:10535000A104B10420F4C4018F519D4FE3D4D701BF
:1053600014968C93BFEFEB1AFB0AEFEF8E1A9E0A8E
:10537000AE0ABE0AE4CF8091400290914102892B8F
:1053800009F483CF8C818D3108F07FCF882E912C4A
:10539000A12CB12CCA80DB80DC24CD24DC24E12CC0
:1053A000F12C8E010F5F1F4F412C512C32014814FC
:1053B00059046A047B0408F068CFFFE1CF16F1E0DE
:1053C000DF06E104F10438F4D80114966C91C601AB
:1053D0008F519D4FC3D4BFEF4B1A5B0A6B0A7B0AF8
:1053E000EFEFCE1ADE0AEE0AFE0A0F5F1F4FDFCF85
:1053F0000E94C8134ACF84E08BCF8C818D3108F096
:1054000044CF882E912CA12CB12CCA80DB80DC24C7
:10541000CD24DC24E12CF12C412C512C32018E01C5
:105420000B5F1F4F481459046A047B0408F02DCF0A
:1054300080E0F0E4CF16F2E0DF06E104F10418F4B6
:10544000C60189966FD4D8018D938D01BFEF4B1A99
:105450005B0A6B0A7B0AEFEFCE1ADE0AEE0AFE0A3F
:10546000E1CF2C81022F10E02D3108F00ECF8A8180
:105470009B819827892798272C01612C712C8034D7
:10548000F2E09F0708F001CF822E912CA12CB12CC5
:1054900040E452E060E070E044195509660977097C
:1054A000421751056105710508F4EFCE20914002C5
:1054B00030914102232B09F03EC01C0129E2220E4B
:1054C000311C80FBEE24FF24E0F880FF0BC088969F
:1054D00029D49D8189279827892781159C4711F414
:1054E0008FEF8D83D501C401840D951DA61DB71DB9
:1054F00080FF19C0680141E0C41AD108CE010596A9
:105500008C0D9D1D9CA78BA7C101800F911F0AD4F4
:10551000ABA5BCA59C9181159C4721F48FEFEBA511
:10552000FCA580838601FE013196EE0DFF1D2FEF55
:10553000E016F10638F08E010F5F1F4FC12CD12C01
:10554000760125C09481858181159C4711F42483BF
:10555000258342E0E40EF11C3296EACF80E448163F
:1055600082E058066104710430F4D80114966C91FD
:10557000C2018996F3D3BFEFCB1ADB0AEB0AFB0A11
:10558000EFEF4E1A5E0A6E0A7E0A0F5F1F4FC814B5
:10559000D904EA04FB0410F378CE80914002909184
:1055A0004102892B09F471CECE0101960E94720A44
:1055B000FFEF21EE34E0F15020403040E1F700C031
:1055C0000000DECC88E0E5E1F1E0DE01919601909B
:1055D0000D928A95E1F7FE0132968FE1DF011D926F
:1055E0008A95E9F786E0898388E07F96DE01159643
:1055F00064CE88E2898381E08A831B821C8245CE47
:105600008B819C81092E000CAA0BBB0B25E0880F17
:10561000991FAA1FBB1F2A95D1F7AC01BD01405E9F
:105620005F4F6F4F7F4F481759076A077B0708F492
:105630002CCE8832E1E09E07A105B10508F025CE09
:105640004932F1E05F076105710520F048E251E061
:1056500060E070E0481B590BBC016A537B4FCE01E0
:1056600001962AD312CE4AE150E06FEF70E0CE01EE
:10567000079641D38091400289830A831B821C8252
:1056800084E08D8386E00CCE81E090E0909346022A
:105690008093450282E390E0909336028093350236
:1056A0000E94AE089093340280933302EECD011530
:1056B000110581F1D0903702C0903B02E090330297
:1056C000F09034020E94AE088E199F09853691052C
:1056D00040F1C6FE26C0D0FE24C00E94AE089093C2
:1056E0003402809333028091350290913602019703
:1056F0009093360280933502892B61F41092460212
:105700001092450281E090E0909341028093400224
:1057100000E010E08091400289830A838091350285
:10572000A4CD82E390E09093360280933502F2CFCD
:105730001092410210924002A8CD0B811C8140E2E0
:1057400050E06FEF70E0CE010196D5D22AEF33E042
:1057500042E050E080E090E0F90165917591061714
:10576000170740F4DE0111968A0F9B1FFC0171831D
:105770006083CA01F4E02A3B3F0709F486CDAC01FF
:105780004E5F5F4F245F3F4F4132510528F37DCD7F
:105790004B815C818AEF93E026EC34E0FC0165915B
:1057A00075916417750709F497C00C962817390787
:1057B000A9F757CD8B819C810AEF13E0F801259161
:1057C00035918217930709F498C0045F1F4FF4E0E6
:1057D000063C1F0799F7EE24EA94FE2CA9C00E940C
:1057E000731053CD8B81853081F0863059F1811152
:1057F0004CCD8FE1FE013196DF011D928A95E9F7CC
:1058000088E08B8383E088A340CD2C816AE0CE01C1
:105810008196FC01362F11923A95E9F7283080F4F1
:10582000629FB00111246F567D4F4AE050E06AD26A
:1058300080E089838AE0FE01B196DE0112963DCDBB
:105840008FEFF7CF6C818AE0FE013596DE019196ED
:1058500001900D928A95E1F78BA19CA181154CE7EF
:10586000940741F42091400230914102232B11F41E
:1058700080E090E09CA38BA38FEF683060F48AE017
:10588000689FB00111246F567D4F4AE050E0CE0171
:10589000819682D280E089830E947A11F6CC809131
:1058A0001F02811509F4FACBB0E1B9BDE2E1E9BD0F
:1058B00009B400FEFDCF8091D8008F7D8093D80081
:1058C0008091E00082608093E0008091E00081FDA3
:1058D000FCCF0E94890CE2CBFC01369625913591D4
:1058E0002115310509F4BDCC4FE150E0BE016E5FDA
:1058F0007F4FF90109958983C8CCF8013896259125
:1059000035912115310509F466CF4CE150E0BE0117
:105910006B5F7F4FC801F90109957C01892B41F428
:10592000F8013A9685919591009711F0FC0109953F
:10593000E982ABCC1F921FB61F9211248F939F93C5
:10594000AF93BF9380911E02811113C08091EC012F
:105950009091ED01A091EE01B091EF014196A11D52
:10596000B11D8093EC019093ED01A093EE01B093F3
:10597000EF01BF91AF919F918F911F901FBE1F901C
:10598000189578941F921FB61F9211248F939F939E
:10599000AF93BF938091EC019091ED01A091EE0146
:1059A000B091EF010196A11DB11D8093EC01909380
:1059B000ED01A093EE01B093EF01BF91AF919F91E4
:1059C0008F911F901FBE1F9018951F920F920FB6B8
:1059D0000F9211242F933F934F935F936F937F9375
:1059E0008F939F93AF93BF93EF93FF938091E100C9
:1059F00082FF09C08091E20082FF05C08091E10032
:105A00008B7F8093E1008091DA0080FF24C0809139
:105A1000D80080FF20C08091DA008E7F8093DA006A
:105A20008091D90080FFA9C080E189BD82E189BD54
:105A300009B400FEFDCF81E0809342028091DB013A
:105A4000811109C00E94530A0E94B00A8091E200AD
:105A500084608093E2008091E10080FF1AC0809111
:105A6000E20080FF16C08091E2008E7F8093E2000A
:105A70008091E20080618093E2008091D800806292
:105A80008093D80019BC85E08093420283E0809324
:105A900011018091E10084FF2FC08091E20084FF1A
:105AA0002BC080E189BD82E189BD09B400FEFDCF34
:105AB0008091D8008F7D8093D8008091E1008F7E07
:105AC0008093E1008091E2008F7E8093E2008091DC
:105AD000E20081608093E2008091DA01811509F48F
:105AE00052C084E08093420280914202843009F0E7
:105AF00052C082E0809311018091E10083FF2CC0AD
:105B00008091E20083FF28C08091E100877F80932D
:105B1000E10082E0809342021092DA018091E1007C
:105B20008E7F8093E1008091E2008E7F8093E2007F
:105B30008091E20080618093E20042E060E080E0DA
:105B40000E94800A8091F00088608093F00081E0DC
:105B50008093110180931001FF91EF91BF91AF915C
:105B60009F918F917F916F915F914F913F912F9175
:105B70000F900FBE0F901F90189519BC1092420203
:105B80001092DB0168CF8091E30087FF02C083E0C1
:105B9000A9CF81E0A7CF81E0ADCF1F920F920FB6C2
:105BA0000F921124EF92FF920F931F932F933F9325
:105BB0004F935F936F937F938F939F93AF93BF9315
:105BC000CF93EF93FF9309EE10E0F8018081C0912D
:105BD000EC008F70C795CC27C795C82B108280EF3B
:105BE000E82EF12CF7018081877F808378940E94D2
:105BF000F00CF8011082F701808188608083CF70FB
:105C0000F801C083FF91EF91CF91BF91AF919F9128
:105C10008F917F916F915F914F913F912F911F9144
:105C20000F91FF90EF900F900FBE0F901F9018955F
:105C30002F923F924F925F926F927F928F929F929C
:105C4000AF92BF92CF92DF92EF92FF920F931F938A
:105C5000CF93DF93CDB7DEB7CA1BDB0B0FB6F8943B
:105C6000DEBF0FBECDBF09942A88398848885F847B
:105C70006E847D848C849B84AA84B984C884DF80EC
:105C8000EE80FD800C811B81AA81B981CE0FD11DD0
:105C90000FB6F894DEBF0FBECDBFED010895EE0F35
:105CA000FF1F0590F491E02D099469279627692735
:105CB0007827872778270895FB01DC0102C005902B
:105CC0000D9241505040D8F70895FB01DC0104C00B
:105CD0008D910190801921F441505040C8F7881BE4
:105CE000990B0895FB01DC0102C001900D92415017
:105CF0005040D8F70895DC0101C06D9341505040E9
:105D0000E0F70895DC01CB01FC01F999FECF06C054
:105D1000F2BDE1BDF89A319600B40D924150504069
:105D2000B8F70895F999FECF92BD81BDF89A9927E9
:105D300080B50895A8E1B0E042E050E0E5CFDC0195
:105D4000A40FB51F4150504040F0CB01840F951F68
:105D50002E9105D041505040D8F70895262FF9993B
:105D6000FECF92BD81BDF89A019700B4021639F0BA
:105D70001FBA20BD0FB6F894FA9AF99A0FBE08958B
:105D80000396272FECDFEADF252FE9DF242FE7CF6B
:105D90000196272FE4DFE2CFDC01CB0102C02D9179
:105DA00005D041505040D8F70895262FF999FECFDD
:105DB0001FBA92BD81BD20BD0FB6F894FA9AF99A28
:105DC0000FBE01960895F894FFCFCD0DF30DF90D98
:105DD000F30DF90D4B0E6C0EF90D720F7F0F711450
:105DE000681483146614D014D0146614D014D0141C
:105DF0009F14D014AA14B514D014D014D014D014F5
:105E00006614D014D0146614D0149114D014D01485
:105E1000CE14CE14CE14CE14CE14CE14CE14CE1472
:105E2000CE14C014D01471146514D014D014D0142E
:105E3000D014D014D014D014D014D014D014C01452
:105E4000D014D0146614D014C614C614C614C614C4
:105E5000C614C614C614C614C614C014D21C3A1DE7
:105E6000DA1CA41CA81CDE1CAC1CE21CEE1CB81C1A
:105E7000331DBC1CF21CC01CF61C1B1DC41CFA1CD0
:105E8000221DCA1C001D081DB01CE61CB41CEA1C07
:105E9000CE1C041D121D2B1D311D9E1CD61C411D28
:105EA0007F1C831C761C7B1C871C8B1C8F1CE22A8E
:105EB000F92A002B45294529332B442B572B982BA6
:105EC0009D2BC82BDA2BEF2BF22B33293729622994
:105ED0006E29792984293129312931293129CD2A7D
:105EE00087298A298E29BB29F829FB29FD29312AEE
:105EF000AB08790B8F0BA909940B700BAF00000056
:105F00000100010101ADE8C35E2B3E72B2004422E4
:105F10006D3B011901AC0041025A027A026694906D
:105F200034C6979192933536323331F7F6F5E20065
:105F3000E900EA00B500B600B700CD008301CC004F
:105F40008A019201940121022302240225022602E1
:105F500027022A02B300B4006F0070009F01CB013A
:105F60009F02A002E200E900EA00B500B600B70017
:105F7000CD008301CC008A01920194012102230209
:105F800024022502260227022A02B300B4006F0071
:0A5F900070009F01CB019F02A002E8
:00000001FF
